:09FCDB00011100010C00010B00F5
:10FC430012F90612FD4F12FDC9E50CB4FF14E518B5
:10FC5300D39400400DD5180AE47833F67F0AFE12D8
:10FC6300FDAC7837E6600712FC80E47837F620B005
:0DFC7300087837E6700312FA35050C80C9D9
:10F90600C2D97580FF43BF027B007A0079087F0069
:10F916007EEE12FDA0AD08E4FFFE12FD937B007A99
:10F926000079097F017EEE12FDA0AD097F017E0000
:10F9360012FD937B007A0079127F027EEE12FDA003
:10F94600AD127F027E0012FD937B007A0079137F51
:10F95600037EEE12FDA0AD137F037E0012FD937BA6
:10F96600007A0079107F047EEE12FDA0AD107F04B0
:10F976007E0012FD937B007A00790E7F057EEE12E3
:10F98600FDA0AD0E7F057E0012FD937B007A007907
:10F996001A7F067EEE12FDA0AD1A7F067E0012FDCE
:10F9A600937B007A0079147F077EEE12FDA0AD14DA
:10F9B6007F077E0012FD937B007A00790A7F087E1E
:10F9C600EE12FDA0AD0A7F087E0012FD937B007A41
:10F9D60000790D7F097EEE12FDA0AD0D7F097E0038
:10F9E60012FD937D1F7F0B7E0012FD937B007A0034
:10F9F600790F7F107EEE12FDA0AD0F7F107E0012F4
:10FA0600FD93E5D85408F522E50FB47F0512FDC92C
:10FA16008011E522B408050202008007E522600392
:0FFA2600020200758081C2B7C2B5D2B6C2B22249
:04FDC900759FA72259
:0BFDAC00EF1FAC0670011E4C70F62229
:10F28C0000C1814001C0804101C0804100C181406A
:10F29C0001C0804100C1814000C1814001C080415A
:10F2AC0001C0804100C1814000C1814001C080414A
:10F2BC0000C1814001C0804101C0804100C181403A
:10F2CC0001C0804100C1814000C1814001C080412A
:10F2DC0000C1814001C0804101C0804100C181401A
:10F2EC0000C1814001C0804101C0804100C181400A
:10F2FC0001C0804100C1814000C1814001C08041FA
:10F30C0001C0804100C1814000C1814001C08041E9
:10F31C0000C1814001C0804101C0804100C18140D9
:10F32C0000C1814001C0804101C0804100C18140C9
:10F33C0001C0804100C1814000C1814001C08041B9
:10F34C0000C1814001C0804101C0804100C18140A9
:10F35C0001C0804100C1814000C1814001C0804199
:10F36C0001C0804100C1814000C1814001C0804189
:10F37C0000C1814001C0804101C0804100C1814079
:10F38C0000C0C101C30302C2C60607C705C5C40439
:10F39C00CC0C0DCD0FCFCE0E0ACACB0BC90908C8A9
:10F3AC00D81819D91BDBDA1A1EDEDF1FDD1D1CDC99
:10F3BC0014D4D515D71716D6D21213D311D1D01009
:10F3CC00F03031F133F3F23236F6F737F53534F4F9
:10F3DC003CFCFD3DFF3F3EFEFA3A3BFB39F9F83869
:10F3EC0028E8E929EB2B2AEAEE2E2FEF2DEDEC2C59
:10F3FC00E42425E527E7E62622E2E323E12120E0C9
:10F40C00A06061A163A3A26266A6A767A56564A4B8
:10F41C006CACAD6DAF6F6EAEAA6A6BAB69A9A86828
:10F42C0078B8B979BB7B7ABABE7E7FBF7DBDBC7C18
:10F43C00B47475B577B7B67672B2B373B17170B088
:10F44C005090915193535292965657975595945478
:10F45C009C5C5D9D5F9F9E5E5A9A9B5B99595898E8
:10F46C00884849894B8B8A4A4E8E8F4F8D4D4C8CD8
:10F47C004484854587474686824243834181804048
:10FCE4000115FF011C0101330001169601380001C2
:05FCF4003400011A00BC
:10FD4F00C2D8E47833F67837F6E51A6003B4FF03C8
:04FD5F00751AFE22F1
:0DFD8600C2D8E47833F67837F67516962269
:09FDB700D2D87F0A7E0002FDACE7
:10FA3500E4F520D2087F04FE12FDACC208A2B09204
:10FA450000D2087F037E0012FDACC208A2B092016D
:10FA5500D2087F037E0012FDACC208A2B09202D28A
:10FA6500087F037E0012FDACC208A2B09203D20843
:10FA75007F037E0012FDACC208A2B09204D2087FBB
:10FA8500037E0012FDACC208A2B09205D2087F0326
:10FA95007E0012FDACC208A2B09206D2087F037E9A
:10FAA5000012FDACC208A2B09207D2087833E6C3B3
:10FAB50094965007E6062439F8A620C2087833E65E
:10FAC500FFB516057837760122EF64077020783A7E
:10FAD500E6FE64036004EEB4060475160822EEB46F
:10FAE5001008783FE62409F5162275169622EFB41C
:10FAF500010475181922EFB40309783AE6B419031D
:04FB05007516062249
:10FCB1007832E6FF7E15D208C2B1DEFEE4FDEF1315
:10FCC10092B1EFC313FF7E12DEFE0DBD08F0D2B17B
:0AFCD1007F087E0012FDACC208227D
:10FC800012F7D5500C12FDB712FDC012F48C12F60B
:10FC90006212FD86E515B40117E4FD7F107EEE12B9
:10FCA000FCFEAD1A7F067EEF12FCFE759F8080FE83
:01FCB0002231
:10F7D5007833E665166002C3227839E6FFF4600ADD
:10F7E500EF651A6005EF6002C322783AE664197086
:10F7F5007AFB7A0079397D0412FBBF8E228F23783C
:10F805003DE6FE08E67C002400FFEC3EFEEF6523A6
:10F815007003EE65226002C322783CE6FF18E6FE1F
:10F82500C39F4004AD078002AD06EEC39F4004AF01
:10F83500068000E51AC39D4006E51AD39F4002C322
:10F8450022AF0C7E0012FC3912FC027C007D1E12D8
:10F85500FB348D25E4F524E524C39525500B7F6401
:10F865007E0012FDAC052480EED322783AE6FF64D3
:10F8750003600CEF64066007EF64106002C3227832
:10F885003BE6FE08E67C002400FFEC3EFEEF640A42
:10F895004E703B783AE6B4030C12FC027C007D0501
:10F8A50012FB348D1BE51B64016002C32212FC02AE
:10F8B5007C007D1412FB348D25E4F524E524C395E5
:10F8C50025500B7F647E0012FDAC052480EE7B0085
:10F8D5007A007939E51624FEFD12FBBF8E228F23AF
:10F8E50074372516F8E6FE74382516F8E67C0024EC
:06F8F50000FFEC3EFEEFF7
:0BF8FB00B52306EEB52202D322C32283
:10F66200E4F525783AE6B4061AE4F5257439252539
:10F67200F8E6FF12FCB512FDC90525E525C394087D
:10F6820040EA22783AE66403600302F76808E6FE7D
:10F6920008E67C002400F523EC3EF522783EE6F5F0
:10F6A200247839E6FF12FCB57839E6FF12FD397885
:10F6B2003AE6FF12FCB5783AE6FF12FD39E5242559
:10F6C200E0FF12FCB5E52425E0FF12FD39E525C374
:10F6D2009524400302F75BE4FF12FCB5E4FF12FD40
:10F6E20039E51CB47B167E00E5232525FFEE352285
:10F6F200FE7B007A00792612FDA0804E7E00E52373
:10F702002525FFEE3522FEC3EF940CEE9400500B3C
:10F712007B007A00792612FD63802F7E00E5232587
:10F7220025FFEE3522FEEF64204E700585BF268050
:10F7320019EF642D4E7005851C26800EEF64304E45
:10F7420070058517268003752601AF2612FCB5AF1A
:10F752002612FD39052502F6CF12FCB17835E6FFF7
:10F7620012FCB502FDC9783AE66410702CF52574D6
:10F77200392525F8E6FF12FCB574392525F8E6FF90
:10F7820012FD390525E525C3940640E312FCB17844
:10F7920035E6FF12FCB502FDC9783AE6641970320B
:03F7A20018E6FF67
:10F7A50012FCB57839E6FF12FD39783AE6FF12FC0E
:10F7B500B5783AE6FF12FD39AF1A12FCB5AF1A1249
:10F7C500FD3912FCB17835E6FF12FCB512FDC922F0
:10F48C00783AE664067064783CE6FFB406117E00B8
:10F49C00783EE6FD12FD93783EE6F51A02F5EA7821
:10F4AC003CE6B40A1CE51B6401600302F5EA783EF5
:10F4BC00E6FD7F067E0012FD93783EE6F51A02F516
:10F4CC00EA783CE6FFB410117E00783EE6FD12FDB2
:10F4DC0093783EE6F51502F5EA783CE6642D600378
:10F4EC0002F5EA783EE6F51C02F5EA783AE6641095
:10F4FC00600302F5EA783EE6F52A08E6FD783BE67D
:10F50C00FCFE08E6F97A002400F525EA3EF5248C89
:10F51C00288929E52A6D7033F526F527C3E527954B
:10F52C002AE5269400505A74402527F8E6F523E581
:10F53C00252527FFE5243526FEAD2312FCFE12FD02
:10F54C00C90527E52770D5052680D1E4F526F527D2
:10F55C00C3E527952AE52694005026E52725E024C7
:10F56C0041F8E6F523E5252527FFE5243526FEADF4
:10F57C002312FCFE12FDC90527E52770D305268052
:10F58C00CF783806E6640870557834E675F002A436
:10F59C002411FFE5F034EEFEE4FD12FCFE7834E6B7
:10F5AC0075F002A42412FFE5F034EEFEE4FD12FC2B
:10F5BC00FE783406E675F002A42411FFE5F034EE73
:10F5CC00FEAD2812FCFE7834E675F002A42412FF7E
:10F5DC00E5F034EEFEAD2912FCFEE47838F6E515C4
:10F5EC00B47F0EE47838F67834F675157E7580F1B4
:10F5FC0022E515B43F1BE4F522AF2212FD2112FDCA
:10F60C00C90522E522C3946440EF75153E75808FC1
:10F61C0022E515B4330D12FDC912FD76751534753E
:10F62C00800F22E515B41F2512FDC97D1F7F107EAA
:10F63C00EE12FCFE7DF07F117EEE12FCFE7DF07F63
:10F64C00127EEE12FCFE75151E75808122E515B436
:06F65C00010312FDC922AA
:09FDC000783576FF783276FF22D7
:10FD39007832E66FFF90F28C937835667932F7EF77
:06FD490090F38C93F622FA
:10FBBF008B268A2789288D29752A00752BFF7DFFB3
:10FBCF00AF291529EF6026AB260528E528AA27704F
:10FBDF0002052714F912FB09652BFF90F28C936D28
:10FBEF00752A00F52BEF90F38C93FD80D3E52BFE58
:03FBFF00EDFF22F5
:04FCF90041000000C6
:10FCFE008E2B8F2C8D2D12FDC975F65575F6AA75A6
:10FD0E00F65575BF04852DF6E52BF5F4852CF575A6
:03FD1E00F7802249
:10FD210075F65575F6AA75F65575BF04EF25E0F51C
:08FD3100F4E4F5F575F78222F8
:10FD760075F65575F6AA75F65575BF0475F783229F
:0BFDA0008F828E83E49312FB227F0110
:01FDAB002235
:0DFD930074002FF582E43400F583EDF022BA
:10FD630074002FF582E43400F583E012FB2212FBCA
:03FD730009FF2263
:01F000001FF0
:0300000002F20009
:0CF20000787FE4F6D8FD7581CE02F2475D
:10FB0900BB010689828A83E0225002E722BBFE02FA
:09FB1900E32289828A83E493222D
:10FB2200BB010689828A83F0225002F722BBFE01C2
:02FB3200F322BC
:10FB3400C2D5EC30E709B2D5E4C39DFDE49CFCEEEC
:10FB440030E715B2D5E4C39FFFE49EFE12FB6AC3FF
:10FB5400E49DFDE49CFC800312FB6A30D507C3E4FA
:06FB64009FFFE49EFE225B
:10FC0200AC2EAD2FAE30AF31780FEFA2E2EC20E692
:10FC120001B35D5E5FF47004FCFDFEFFEF13FFEEC7
:10FC220013FEED13FDEC13FCD8E08C2E8D2F8E30DD
:10FC32008F31EE547FFE228E2E8F2FE4F530F53178
:01FC4200229F
:10F20C0002FC43E493A3F8E493A34003F68001F2D9
:10F21C0008DFF48029E493A3F85407240CC8C33303
:10F22C00C4540F4420C8834004F456800146F6DFD2
:10F23C00E4800B010204081020408090FCDBE47E8B
:10F24C00019360BCA3FF543F30E509541FFEE493C7
:10F25C00A360010ECF54C025E060A840B8E493A38E
:10F26C00FAE493A3F8E493A3C8C582C8CAC583CAB9
:10F27C00F0A3C8C582C8CAC583CADFE9DEE780BE71
:01FCFD000006
:10FB6A00BC000BBE0029EF8DF084FFADF022E4CC7F
:10FB7A00F875F008EF2FFFEE33FEEC33FCEE9DEC48
:10FB8A00984005FCEE9DFE0FD5F0E9E4CEFD22ED8E
:10FB9A00F8F5F0EE8420D21CFEADF075F008EF2FD8
:10FBAA00FFED33FD4007985006D5F0F222C398FDC9
:05FBBA000FD5F0EA2266
:00000001FF
